:020000040000FA
:0600000060283E300130D3
:08000800A000030EA100831209
:1000100005191028831601178312B2308100422877
:100020008316011383120B191C28AE17280A031913
:100030002E17AE192D283B28AE13AE192A282E1FD5
:100040003B28AE1A3B28A701A601A501A801AE01D5
:10005000AE164228F030AE0542282D152E13AE12F2
:100060002708AB002608AA002508A9002808AC002C
:10007000F030AE0542282E0DA80DA50DA60DA70D3A
:10008000AE1AAE0A8B100B11210E8300A00E200EAB
:02009000090065
:1000C000203084008001840A60300402031C62280E
:1000D000B8228316FF239000831283160C30850507
:1000E000870183128501870107309900003083164C
:1000F00091009F008312C830831681008312313033
:100100009000003083168C00831210308B00BD1BD2
:100110008B28851D3D233D1BBE013D1BBF013D1F9F
:10012000262381018E018F010B118B100B108C1374
:100130000C138C110C108B17AD202D19AF208C22B5
:10014000B30BAA28031085190314BA0DF0303A0234
:100150000319E321BD1865239C28640008002908C1
:100160003F3C0319BB282B082A0629062C02031D35
:100170002D11031D08002D110130B7008B13203005
:10018000370783169B001C141A088312A400103032
:10019000370783169B001C141A088312A300003033
:1001A000370783169B001C141A088312A2008B17B2
:1001B00024082B02031DDD2923082A02031DDD2943
:1001C000013009303702031D132929083F3C031968
:1001D000FD2840302906E039031DF3283F1FF3288E
:1001E0003F13AD17012960302906E039031D0129AD
:1001F0003F1B01293F17AD170129AC1F3F13AC1B53
:100200003F1780302906F039031D0A29BF1F0A292C
:10021000BF13AD1790302906F039031D1329BF1BFA
:100220001329BF17AD17A91FDD29291BDD292208B6
:100230002906F039A91EE039031DDD292208290508
:100240000F3903197D2901303702031D2C293E186F
:100250002C293E14AD17CE2202303702031D35295A
:10026000BE183529BE14AD17D02203303702031D46
:100270003E293E193E293E15AD17D22204303702E1
:10028000031D4729BE194729BE15AD17D4220530D5
:100290003702031D50293E1A50293E16AD17D622AB
:1002A00006303702031D5929BE1A5929BE16AD174B
:1002B000D82207303702031D62293E1B62293E17F0
:1002C000AD17DA2208303702031D6B29BE1B6B29DC
:1002D000BE17AD17DC2209303702031D74293F1801
:1002E00074293F14AD17DE220A303702031D7D2921
:1002F000BF187D29BF14AD17E222290922050F3945
:100300000319DD2901303702031D8B293E1C8B297F
:100310003E10AD17E62202303702031D9429BE1CA1
:100320009429BE10AD17E82203303702031D9D2922
:100330003E1D9D293E11AD17EA2204303702031DF0
:10034000A629BE1DA629BE11AD17EC220530370225
:10035000031DAF293E1EAF293E12AD17EE22063017
:100360003702031DB829BE1EB829BE12AD17F022F0
:1003700007303702031DC1293E1FC1293E13AD17A7
:10038000F22208303702031DCA29BE1FCA29BE1334
:10039000AD17F42209303702031DD3293F1CD3299E
:1003A0003F10AD17F6220A303702031DDC29BF1CAF
:1003B000DC29BF10AD17FA22DD29B70A0B3037024E
:1003C00003180800BE28B601B3019630B40001300E
:1003D000B5000130B70085018701AD136C22AD2057
:1003E000B30B2D2A031085190314BA0DF0303A020D
:1003F00003195C2AB40B2D2A013037020319FE229F
:10040000023037020319022303303702031906238F
:100410000430370203190A230530370203190E236B
:100420000630370203191223073037020319162347
:100430000830370203191A230930370203191E2323
:100440000A303702031922233708B6080319B60009
:1004500003192B2AB6039630B4002D1DEF292D1158
:10046000A91FEF29291BEF29A91E29120F302905E1
:100470000319EF29B9012918B90AA918B90A2919C4
:10048000B90AA919B90AB918EF293919EF298B1333
:1004900020303707BC002B08BB009A2210303707EA
:1004A000BC002A08BB009A2200303707BC0029088C
:1004B000BB009A228B17662285018701B70AB60115
:1004C0000B303702031CEF29262308000A303702BD
:1004D00003190800850187011430B90033300F1E5D
:1004E00085000F1A8501FF300F1A87000F1E870144
:1004F000AD202D1D6E2A2D11290A0319832AA91F4B
:100500006E2A291B6E2A0F302905031D6C2AB90B90
:100510006E2A850187010800AD1F0800AD13103059
:10052000BC003E08BB009A223030BC003F08BB0034
:100530009A2208003C088B1383169B001C141A088F
:1005400083128B173B02031908008B133B08831699
:100550001C159A003C089B0055309D00AA309D0058
:100560009C1464009C18B12A1C1183128B1708007C
:10057000831600309B001C141A088312BD008316DA
:1005800010309B001C141A088312BE0083163030F2
:100590009B001C141A088312BF00080005160800EF
:1005A0008516080005140800851408008714080043
:1005B000071508000714080087160800BD18080072
:1005C00007160800BD180800871508000512080066
:1005D0008512080005100800851008008710080023
:1005E000071108000710080087120800BD1808004E
:1005F00007120800BD180800871108000508103A06
:10060000850008000508203A850008000508013A21
:10061000850008000508023A850008000708023A2C
:10062000870008000708043A870008000708013A15
:10063000870008000708203A870008000708103ADA
:10064000870008000708083A870008003E180516CA
:10065000BE1885163E190514BE1985143E1A871456
:10066000BE1A07153E1B0714BE1B8716BD180800CF
:100670003F180716BF1887150800B601B301B4016B
:100680003D1C452B3D10BD14482BC030BD053D140D
:100690003D083F39B60064004D2B4E2B4F2B502B9D
:1006A000512B3330B41B8500B41F8501B30B4B2B8A
:1006B000B40B4B2B0310B60CB608031D4B2B0030AC
:1006C000BC003D08BB009A220800BF1F702B3F1BD7
:1006D00007123F1B87153F1F07163F1F8711080092
:0606E0000712871108005B
:084000000200000006000200AE
:02400E00CC01E3
:1042000001008100820084008800B100B200B40087
:10421000B800A100A200FF00FF00FF00FF00FF00A8
:104220000000010001000100010001000100010087
:10423000010001000100FF00FF00FF00FF00FF0080
:10424000010000000000000000000000000000006D
:10425000000000000000FF00FF00FF00FF00FF0063
:104260000000FF00FF00FF00FF00FF00FF00FF0055
:10427000FF00FF00FF00FF00FF00FF00FF00FF0046
:10428000FF00FF00FF00FF00FF00FF00FF00FF0036
:10429000FF00FF00FF00FF00FF00FF00FF00FF0026
:1042A000FF00FF00FF00FF00FF00FF00FF00FF0016
:1042B000FF00FF00FF00FF00FF00FF00FF00FF0006
:1042C000FF00FF00FF00FF00FF00FF00FF00FF00F6
:1042D000FF00FF00FF00FF00FF00FF00FF00FF00E6
:1042E000FF00FF00FF00FF00FF00FF00FF00FF00D6
:1042F000FF00FF00FF00FF00FF00FF00FF00DD00E8
:00000001FF
